:1000000009298030A100FE30A7200130A7207530DB
:10001000A7003030BE28A101A117AF00AF08031D13
:100020001328030114280130AF020310A20CA20C04
:10003000A20CC0302205403EAF07FE30A7202F089B
:10004000A728A101A117AF00FE30A7202F08A728DD
:10005000A401AA00AB01A01124080319A0150530C2
:10006000A3002730A900103041200330A900E83058
:100070004120A90164304120A9010A3041202A0809
:100080004828A8002B08A7002A08A600D220260886
:10009000A600A3030319A011240803195228230260
:1000A000031859282608031DA011A0195928303E0D
:1000B000A7280800AD0006118611831606118611C7
:1000C0000F30860583122D08A01884283E30A70023
:1000D0008030BE203330AC0098201330A700883029
:1000E000BE2098206430BD2098206430BD2022308E
:1000F000AC009820283083200C30832006308320E9
:10010000A0142D0884282014AC00201C92288611ED
:10011000033C031C972897200530A700DC30BE2045
:10012000031408002014FE3C0319A5288615201C82
:10013000201006150F3086052C08F03986040611AC
:10014000AC0E201898283230BD202D080429A11BA0
:100150005A2883178001840AFF3E031DAA28042918
:10016000A901A800FF30A807031CA907031C042944
:100170000330A700DF30BE20B228A701E83EA6006A
:10018000A709FC30031CC728A6070318C428A60724
:100190000000A70FC4282618CD28A61CD1280000CF
:1001A000D1280800AB01AA011030AC00270DAA0D20
:1001B000AB0D2808AA022908031C290FAB0203185B
:1001C000E8282808AA0729080318290FAB070310F5
:1001D000A60DA70DAC0BD628260804291030B000B8
:1001E000A701A601AD0CAC0C031CFC282808A6072F
:1001F00029080318290FA707A70CA60CAB0CAA0CFB
:10020000B00BF2282A080429831383120313000079
:100210000800A00107309F00E03083168500FF3002
:1002200086008113831285018601203084006030AE
:10023000AA20A03084005030AA2020308400303022
:10024000A920C830B020012077305A205A205A20E7
:100250002E305A2070305A2069305A2063305A208C
:1002600062305A2061305A2073305A2069305A2047
:1002700063305A202E305A206E305A206C305A206B
:100280000B30A900B830B120012044305A2043304F
:100290005A2046305A2032305A2030305A204E30C0
:1002A0005A204C305A2042305A2020305A205A20AE
:1002B00056305A202D305A2032305A200730A900AB
:1002C000D030B12001204C305A2044305A205230D6
:1002D0005A2020305A2061305A2066305A2072301D
:1002E0005A2065305A2067305A2065305A206C30C9
:1002F0005A2065305A206E305A2086188529851F6D
:1003000083290514842905107D29012053305A20A2
:1003100069305A2067305A206E305A2061305A2096
:100320005A206C305A2020305A207A305A206F30B0
:100330005A2065305A206B305A2065305A206E3072
:100340005A2036140512831605128312342AC3016B
:100350003C03A500C90149082502031CC029E3216B
:10036000B61CBE294308A6004908A200A601A20A9D
:100370000314A60DA20BB9292608C304C90FAB2983
:10038000B2014308B100B20CB10CB20CB10CB20C0A
:10039000B10CB20CB10C0F30B2053208AD0031080F
:1003A000AC00A9010A30A800EE20B1002B08B20071
:1003B000B4014308B3000F30B3050030B405310871
:1003C0003307C3000800BA01B9010618F829013043
:1003D000B020B90A0319BA0A0B303A02031CF729F4
:1003E000031DF629B9303902031CF729812CE529B0
:1003F0009B30B0200618B614061CB610361C142A02
:10040000AD014408AC00A9011430A800EE20B100F1
:100410002B08B2003208A7003108A600A9013A3023
:10042000A800D220BD00272A8030A1000130A20000
:100430003D080D200230A40044082920030136198C
:10044000013EB618013A03193611031D3615C40AC8
:1004500085140130A900F430B1208510A901F030D5
:10046000A8002808B1200800BB01C4013612361AC2
:10047000D12ABA01B901061C4E2AB90A0319BA0ACF
:100480000130B020AF303A02031C4D2A031D4C2A24
:10049000C9303902031C4D2A812C3B2ABA01B9010B
:1004A00006188A2AB90A0319BA0A0A30B02036187F
:1004B0007E2A39080B3A3A04031D692A8030A100CC
:1004C0000130A2003D080D2035305A2039305A2025
:1004D0007D2A3908193A3A04031D702A85147D2AA9
:1004E00039084B3A3A04031D772A85107D2A3908CA
:1004F000FA3A3A04031D7D2A812C892A11303A02E6
:10050000031C892A031D882A95303902031C892A75
:10051000812C502A41303B02031C8F2A812CBB0ABC
:100520003A08031D972A65303902031C982A3616AB
:10053000361CD02AAD013B08AC00A9011430A8003C
:10054000EE20B1002B08B2003208A7003108A60047
:10055000A9014130A800D220BD008030A100803028
:10056000212053305A2069305A2067305A206E308B
:100570005A2061305A205A206C305A2020305A209C
:1005800067305A2065305A2076305A206F305A2012
:100590006E305A2064305A2065305A206E305A200E
:1005A000372A361CF32A012049305A206E305A204F
:1005B00069305A2074305A2069305A2061305A20EC
:1005C0006C305A2069305A2073305A2065305A20D6
:1005D00072305A2065305A206E305A202E305A2000
:1005E0005A205A20622B0B30BD000130A2003D087A
:1005F0000B20A101B61D0B2B3B3041020318022B2F
:10060000C10A0A2BC101173045020318092BC50A7C
:100610000A2BC5010F2B4208C1004608C500051B67
:100620001F2B4508031D172B0C30C7001E2B0D3048
:100630004502031C1E2B0C304502C700242B450825
:10064000C70020305A205A200A30470203182A2BAC
:1006500020305A208030A100470828203A305A2004
:100660000230A400410829203A305A2030305A2064
:100670005A20051B4B2B0C3045020318442B6130CC
:100680005A206D305A20482B70305A206D305A2035
:100690001130BD004D2B1330BD004108031901304E
:1006A000031D0301B5001E30410203190130031D73
:1006B00003013504B5000130861803013504031920
:1006C000622B592C361E572CE3210130C9000F3004
:1006D000490203186E2BE321C90F672B3611B6119F
:1006E000E321E321E321B61C772B0514782B0510B9
:1006F0001230C900143049020318812BE321C90FBD
:100700007A2BE3210730BC00A7214308C200E32174
:10071000361D8B2BB6150630BC00A7214308C6003A
:10072000E321361D942BB6150630BC00A7214308E3
:10073000BE000330BC00A7214308C8000530BC0040
:10074000A7214308C0000830BC00A7214308BF0010
:10075000E321361DAC2BB615361CB22BB619B12BC6
:1007600036100120B619562C8030A100803021208F
:100770003E08282020305A2001304002031DC72B9C
:100780006A305A2061305A206E305A203F2C023095
:100790004002031DD22B66305A2065305A20623049
:1007A0005A203F2C03304002031DDD2B6D305A20B0
:1007B00072305A2074305A203F2C04304002031DFE
:1007C000E82B61305A2070305A2072305A203F2C6A
:1007D00005304002031DF32B6D305A2065305A203E
:1007E00069305A203F2C06304002031DFE2B6A3030
:1007F0005A2075305A206E305A203F2C0730400264
:10080000031D092C6A305A2075305A206C305A204A
:100810003F2C08304002031D142C61305A207530E3
:100820005A2067305A203F2C09304002031D1F2CEC
:1008300073305A2065305A2070305A203F2C0A30CD
:100840004002031D2A2C6F305A206B305A2074301E
:100850005A203F2C0B304002031D352C6E305A209D
:100860006F305A2076305A203F2C0C304002031D46
:100870003F2C64305A2065305A2063305A20051BC3
:100880004C2C20305A208030A1000230A4003F08B8
:10089000292020305A20562C20305A2027305A2028
:1008A0008030A1000230A4003F082920582C812C60
:1008B000342A851F602C0512831605128312622CC0
:1008C0008316051683129B30B020410803190130AE
:1008D000031D0301B5000130861803013504031917
:1008E000722C0515851585140130A900F430B1204E
:1008F0000511851185100130A9004A30B120C40AC4
:10090000652B012047305A2065305A205A206E301E
:100910005A2020305A2073305A2069305A206730CC
:100920005A206E305A2061305A205A206C305A209A
:10093000203084006030AA20A03084005030AA20EB
:10094000203084003030A9200618B616061CB612D6
:1009500003010618013EB61A013C031DB52CB70A67
:100960000319B80A0130B020A82C0301B61A0130CF
:10097000013A0319B612031DB61603010618013E0B
:10098000B61A013C031DCA2CB70A0319B80A013074
:10099000B020BD2C03303802DE30031937020318B3
:0609A000982C3614342AE5
:02400E00503F21
:00000001FF
